:10000000830100308A008928F70003088301C600B5
:100010000408C7000A08C8008A01831203130C1CD5
:100020001228132825280C10201C172818282028EF
:100030003208F93E8F0031088E000716201025285F
:100040000712B8308F008E0120148C1C2828292814
:100050002A288C108C1E2D282E2880281808C500D0
:10006000C51C332834283F28071018121A08C50069
:100070001A08C5001A08C500AF0107147F28451DDE
:10008000422843284A2887121A08C5001812AF01CF
:1000900087167F287B281A08C50045083A3A031DB1
:1000A000522853285428AF0145080D3A03195928FE
:1000B0005E2845083A3A03195F285E2861286028BF
:1000C00068282F08A03E8400831345088000AF0AEB
:1000D00045080D3A031D6D286E287B282F08A03E89
:1000E00084008313450880002F0AA03E84008313F8
:1000F0008001AF01A0148C1A7E287F284B28181687
:100100004708840048088A0046088300F70E770EE7
:1001100009002030840021309C20213084004630AA
:100120009C20A0308400DC309C2083010A128A11BC
:10013000462C04068001840A040603190034992819
:1001400083120313C900CA1BAE284A1BB6284A08EB
:100150008A004908C90A0319CA0A820083134A1887
:1001600083174908C90A840000080800543457342A
:100170000D340034543443340D3400344334523499
:100180002034313438342034333432342034313470
:1001900039342034333432340D3400344C34313477
:1001A000203432340D3400344D344D342034313465
:0601B00030340D34003470
:1002940000300A128A11BA2DF0000030711870076C
:1002A4000310F00D0310F10CF10803190800502994
:1002B40083120313BD003A303D0203186429303021
:1002C4003D0208000310080005308316031399004B
:1002D4002430980090308312980083168C16831271
:1002E400080083120313C4007829782983120313A6
:1002F4000C1E7D297E29772944089900812908004C
:10030400F401F5010310F30CF20C031C902970089E
:10031400F40771080318710AF5070310F00DF10DC5
:100324007208730403190034842983120313B6007A
:100334000230B7003F30B800A029A029B80BA32988
:10034400A4299F29B70BA729A8299C29B60BAB2957
:10035400AC299A290800831203133808BA00390813
:10036400BB003B08CA003A08BA0A0319BB0A0A12BE
:100374008A11A0200A128A110038031DB3293B08F0
:10038400F1003A08F0003808F002031CF1033908C0
:10039400F102FF30F007031CF1070800D429B80A62
:1003A4000319B90A831203133908CA0038080A1258
:1003B4008A11A0200A128A11203A0319D129390876
:1003C400CA0038080A128A11A0200A128A11093AAE
:1003D4000319D129BB01BC01BA013908CA00380884
:1003E4000A128A11A0200A128A112D3A031DFC292F
:0C03F400BA0A072A3908CA0038080A12A1
:100400008A11A0200A128A112B3A031D0A2AB80A5F
:100410000319B90A3908CA0038080A128A11A0203B
:100420000A128A115A210A128A11031C3A2A0A3026
:10043000F200F3013C08F1003B08F0000A128A11B7
:1004400082213908CA0038080A128A11A0200A122B
:100450008A11F000F1017408F0070318F10A750819
:10046000F107D0307007BB00FF3003180030710770
:10047000BC00072ABA080319472A3C08F1003B08C8
:10048000F000F009F109F00A0319F10A08003C082C
:10049000F1003B08F0000800A23083120313B800FB
:1004A0008030B9000A128A11D0210A128A1170080C
:1004B000B000A030B8008030B9000A128A11AD2116
:1004C0000A128A117008B6000330B700682AB70A0A
:1004D0003708A03E840083130008203A031D712AC8
:1004E000762A36083702031C772A762A792A782A50
:1004F000672A3708A03EB8008030B9000A128A1176
:10050000D0210A128A117008A600B70A882AB70AF1
:100510003708A03E840083130008203A031D912A67
:10052000962A36083702031C972A962A992A982A6F
:10053000872A3708A03EB8008030B9000A128A1115
:10054000D0210A128A117008A400B70AA82AB70A93
:100550003708A03E840083130008203A031DB12A07
:10056000B62A36083702031CB72AB62AB92AB82A8F
:10057000A72A3708A03EB8008030B9000A128A11B5
:10058000D0210A128A117008A200B70AC82AB70A35
:100590003708A03E840083130008203A031DD12AA7
:1005A000D62A36083702031CD72AD62AD92AD82AAF
:1005B000C72A3708A03EB8008030B9000A128A1155
:1005C000D0210A128A117008A500B70AE82AB70AD2
:1005D0003708A03E840083130008203A031DF12A47
:1005E000F62A36083702031CF72AF62AF92AF82ACF
:1005F000E72A3708A03EB8008030B9000A128A11F5
:10060000D0210A128A117008A300B70A082BB70A72
:100610003708A03E840083130008203A031D112BE5
:10062000162B36083702031C172B162B192B182BE9
:10063000072B3708A03EB8008030B9000A128A1193
:10064000D0210A128A117008A1000800A23083127A
:100650000313B8008030B9000A128A11D0210A129F
:100660008A117008B000A030B8008030B9000A12BA
:100670008A11AD210A128A117008B6000330B70042
:10068000422BB70A3708A03E840083130008203AA3
:10069000031D4B2B502B36083702031C512B502BBC
:1006A000532B522B412B3708A03EB8008030B900A5
:1006B0000A128A11D0210A128A117008A700B70AFB
:1006C000622BB70A3708A03E840083130008203A43
:1006D000031D6B2B702B36083702031C712B702BFC
:1006E000732B722B612B3708A03EB8008030B90005
:1006F0000A128A11D0210A128A117008A800B70ABA
:10070000822BB70A3708A03E840083130008203AE2
:10071000031D8B2B902B36083702031C912B902B3B
:10072000932B922B812B3708A03EB8008030B90064
:100730000A128A11D0210A128A117008A900B70A78
:10074000A22BB70A3708A03E840083130008203A82
:10075000031DAB2BB02B36083702031CB12BB02B7B
:10076000B32BB22BA12B3708A03EB8008030B900C4
:100770000A128A11D0210A128A117008AB00B70A36
:10078000C22BB70A3708A03E840083130008203A22
:10079000031DCB2BD02B36083702031CD12BD02BBB
:1007A000D32BD22BC12B3708A03EB8008030B90024
:1007B0000A128A11D0210A128A117008AA00B70AF7
:1007C000E22BB70A3708A03E840083130008203AC2
:1007D000031DEB2BF02B36083702031CF12BF02BFB
:1007E000F32BF22BE12B3708A03EB8008030B90084
:1007F0000A128A11D0210A128A117008AC00B70AB5
:10080000022CB70A3708A03E840083130008203A60
:10081000031D0B2C102C36083702031C112C102C36
:10082000132C122C012C3708A03EB8008030B900E0
:100830000A128A11D0210A128A117008AE00B70A72
:10084000222CB70A3708A03E840083130008203A00
:10085000031D2B2C302C36083702031C312C302C76
:10086000332C322C212C3708A03EB8008030B90040
:100870000A128A11D0210A128A117008AD002030A4
:100880002D02031C442C452C452C0800FA300A127A
:100890008A1197210A128A110A128A1166210A12F4
:1008A0008A11F13083169200831295019B01831601
:1008B000071187103C30831291003C3097003C3088
:1008C0009D00073092071F10063083169F00850198
:1008D0008312851105118510051001309000B83084
:1008E0008F008E0183160C140B178B1707128711BC
:1008F000803087008312AF01A0102830B100B20110
:10090000831686018312B301852CFA300A128A11EC
:1009100097210A128A11B30A1F303302031C912C4B
:10092000922C852CD430B7000030B8000A128A11FE
:100930004A210A128A11FA300A128A1197210A12E0
:100940008A11CE30B7000030B8000A128A114A214D
:100950000A128A11FA300A128A1197210A128A1190
:10096000BE30B7000030B8000A128A114A210A12BC
:100970008A11FA300A128A1197210A128A11B630A6
:10098000B7000030B8000A128A114A210A128A11EF
:10099000FA300A128A1197210A128A11D930B70047
:1009A0000030B8000A128A114A210A128A11FA305C
:1009B0000A128A1197210A128A11FA300A128A1130
:1009C00097210A128A11BA30B7000030B8000A1213
:1009D0008A114A210A128A11FA300A128A119721C1
:1009E0000A128A11071487168715A01CF82CF92CF7
:1009F000B62D83162008533A031DFF2C002D052D1C
:100A00000A128A114C220A128A11831620084E3AC1
:100A1000031D0B2D0C2D132D0A128A1126230A12E9
:100A20008A11051185118312A01010302D020318B0
:100A30001A2D1B2D4C2D8711051105108511B40A97
:100A40000319B50A003035023C3003193402031C87
:100A50002A2D2B2D312D1E30950005151E30B1008D
:100A6000B20100303502783003193402031C392DED
:100A70003A2D3D2D9630B100B20100303502B43030
:100A800003193402031C452D462D4A2D2C30B1008C
:100A90000130B2008715B62DB401B50142302802ED
:100AA0000318532D542D6A2D003032021E300319C5
:100AB0003102031C5C2D5D2D622DE230B107031C59
:100AC000B2036A2D05148514D2309500D2309B00F4
:100AD000051585154C302802031C6F2D702D7D2DBA
:100AE00002303202ED30031931020318782D792DCE
:100AF0007D2D1430B1070318B20A32302E020318CC
:100B0000882D822D0B302E02031C882D872D8A2DD7
:100B1000892D922D05150510851585101E3095001F
:100B20001E309B0065302E02031C972D982DA02DA2
:100B300005148514D2309500D2309B00051585151B
:100B40005A303002031CA52DA62DAB2D051505101E
:100B5000283095008511293030020318B02DB12DB1
:100B6000B62D8515851028309B000511F52C0A122D
:100B70008A11892883120313BF00BD013608BA0009
:100B8000AE2F3E08253A031D9F2FFF30BB00BC014E
:100B9000B901612FBF080319D12D3F0884008313C9
:100BA00080013D0808000230BA073A02840083132E
:100BB00000089D2FB90AE02D0830BB07FE30BB07A7
:100BC0000230BA073A02840083130008C000840A86
:100BD0000008C1003918C11FF42DC009C109C00A9D
:100BE0000319C10ABC03F52DB9010B30BB073B0843
:100BF000F200F3014108F1004008F0000A128A11E6
:100C0000C6277008BE003B08F200F3014008F00060
:100C10004108F1000A128A11C6270A128A117408C3
:100C2000C0007508C100C201C20AC30143084102E5
:100C3000031D1C2E42084002031C412E3B08F200FB
:100C4000F3014208F0004308F1000A128A118221E0
:100C50000A128A117408C2007508C300BC03162E5C
:100C6000BD0ABF0803193B2E3F08840083132030C0
:100C70008000BF0A412E20300A128A1173210A1205
:100C80008A11BC033C08803A7F3E0318302E391C81
:100C9000582EBD0ABF080319542E3F088400831341
:100CA0002D308000BF0A582E2D300A128A11732170
:100CB0003B08F200F3014208F0004308F1000A1279
:100CC0008A11C6270A128A117408C2007508C30067
:100CD00042040319972E4308F3004208F20041082A
:100CE000F1004008F0000A128A11C6277408F000CB
:100CF0007508F1003B08F200F3010A128A11C627B9
:100D00000A128A117008BC00803A763E031C8A2EB3
:100D10000730BC07BD0ABF080319942E3F088400A2
:100D200083133C08303E512E3C08303E552E0A308D
:100D30003E02031C9D2E0730BE07BD0ABF080319E3
:100D4000A72E3F08840083133E08303EA72F3E089D
:100D5000303EAB2FBD0ABF080319B52E3F088400F3
:100D6000831320308000BF0ABB2E20300A128A1164
:100D700073210A128A11BC033C08803A7E3E031894
:100D8000AA2E0230BA073A02840083130008BE007C
:100D90009F2F0230BA073A02840083130008C20072
:100DA000840A0008C300BE013E084207C900430888
:100DB000CA0049080318CA0A0A128A11A0200A1296
:100DC0008A1100380319E62EBE0AD42E3B083E02D3
:100DD0000318EC2E3E08BB003B08BC1B232FFF3A38
:100DE0003C07031C232FBD0ABF080319FE2E3F0832
:100DF0008400831320308000BF0A042F20300A12A1
:100E00008A1173210A128A11BC03EC2E4308CA000E
:100E100042080A128A11A0200A128A11BE00C20AD0
:100E20000319C30ABD0ABF0803191D2F3F08840018
:100E300083133E088000BF0A232F3E080A128A113E
:100E400073210A128A11BB033B0F062FAE2F3808FD
:100E5000CA0037080A128A11A0200A128A112A3AF7
:100E6000031D392F0230BA073A02840083130008A9
:100E70005D2F3808CA0037080A128A11A020D03E18
:100E8000BB00B70A0319B80A3808CA0037080A12A3
:100E90008A11A0200A128A11BE0030303E02031CC3
:100EA000612F3A303E020318612F0A30F1003B08EF
:100EB0000A128A114E213E07D03EBB00B70A031921
:100EC000B80A3808CA003708B70A0319B80A0A125C
:100ED0008A11A0200A128A11BE00003A0319CA2DF5
:100EE0002A3A0319D32D043A0319272F763A031906
:100EF000DC2D3B3A0319BC2E073A0319DA2D0B3AC5
:100F00000319DE2D1C3A0319C92E063A0319E02DE8
:100F10000D3A0319DC2D30303E02031C9F2F3A306E
:100F20003E0203189F2F0A30F1003C080A128A1172
:100F30004E210A128A113E07D03EBC00612FBD0A25
:100F4000BF080319AA2F3F08840083133E088000BE
:100F5000BF0AAE2F3E080A128A1173213808CA0050
:100F60003708B70A0319B80A0A128A11A0200A1210
:100F70008A11BE00BE08031DC12DBF080319C42F6E
:100F80003F088400831380013D080800F601F40146
:100F9000F50172087304031DD02FF001F101003434
:100FA0001F30F6040310F60AF20DF30D031CD32FC5
:100FB000F30CF20C73087102031DE02F720870022B
:100FC000031CE82F7208F0027308031C730AF10275
:100FD000F40DF50DF60BF61AD82FF61FF42FF409C1
:100FE000F40A0319F503F5097408F2007508F30013
:100FF000761F0034F009F00A0319F103F1090034F7
:02400E00713F00
:00000001FF
